:100000000C9462000C947F000C947F000C947F0091
:100010000C947F000C947F000C947F000C94990149
:100020000C947F000C947F000C947F000C947F0054
:100030000C947F000C947F000C947F000C947F0044
:100040000C944F010C947F000C947F000C947F0063
:100050000C947F000C947F000C947F000C947F0024
:100060000C947F000C947F00000000002300260009
:1000700029000200000000240027002A00000000E0
:1000800000250028002B00040404040404040402D6
:100090000202020202030303030303010204081025
:1000A00020408001020408102001020408102000F2
:1000B0000000080002010000030407000000000027
:1000C0000000000011241FBECFEFD8E0DEBFCDBF7F
:1000D00011E0A0E0B1E0E8E0FCE002C005900D9284
:1000E000A230B107D9F721E0A2E0B1E001C01D9232
:1000F000A032B207E1F70E943A020C9402060C9477
:10010000000090E0FC01E155FF4F2491FC01E55611
:10011000FF4F3491FC01E957FF4FE491EE23C9F002
:10012000222339F0233001F1A8F4213019F12230D3
:1001300029F1F0E0EE0FFF1FE358FF4FA591B491B6
:100140008FB7F894EC91611126C030953E233C9313
:100150008FBF08952730A9F02830C9F0243049F71F
:10016000809180008F7D03C0809180008F77809385
:100170008000DFCF84B58F7784BDDBCF84B58F7DE2
:10018000FBCF8091B0008F778093B000D2CF809169
:10019000B0008F7DF9CF3E2BDACFCF93DF9390E085
:1001A000FC01E556FF4F249189579F4FFC01849134
:1001B0008823D1F090E0880F991FFC01ED58FF4F84
:1001C000A591B491FC01E358FF4FC591D491611101
:1001D0000EC09FB7F8948C91E22FE0958E238C93FC
:1001E0002881E223E8839FBFDF91CF9108958FB7E5
:1001F000F894EC91E22BEC938FBFF6CF3FB7F894D5
:1002000080911C0190911D01A0911E01B0911F01D0
:1002100026B5A89B05C02F3F19F00196A11DB11D61
:100220003FBFBA2FA92F982F8827BC01CD01620F9D
:10023000711D811D911D42E0660F771F881F991F58
:100240004A95D1F708959091000189130BC0E2E718
:10025000F0E0E4919FEF90930001E13049F028F045
:10026000E23061F060E00C94810010926E00FACFF1
:1002700090916F009D7F90936F00F4CF90917000EC
:100280009D7F9093700091E09093B0009091B100A9
:10029000987F94609093B1001092B300E3CF1F92C7
:1002A0000F920FB60F9211242F933F938F939F932A
:1002B000AF93BF938091180190911901A0911A01F9
:1002C000B0911B013091170123E0230F2D3758F512
:1002D0000196A11DB11D20931701809318019093E1
:1002E0001901A0931A01B0931B0180911C019091F8
:1002F0001D01A0911E01B0911F010196A11DB11D0C
:1003000080931C0190931D01A0931E01B0931F01C7
:10031000BF91AF919F918F913F912F910F900FBE01
:100320000F901F90189526E8230F0296A11DB11D6E
:10033000D2CF1F920F920FB60F9211242F933F939B
:100340004F935F936F937F938F939F93AF93BF93DD
:10035000EF93FF938091070190910801A09109010B
:10036000B0910A01892B8A2B8B2BD1F1909102013C
:10037000E0910301F09104018081892780838091BD
:10038000070190910801A0910901B0910A01181686
:1003900019061A061B069CF480910701909108012A
:1003A000A0910901B0910A010197A109B1098093B7
:1003B000070190930801A0930901B0930A01FF91EE
:1003C000EF91BF91AF919F918F917F916F915F91CD
:1003D0004F913F912F910F900FBE0F901F90189546
:1003E000809100010E942301EACFCF92DF92EF9229
:1003F000FF920F931F93E82FF92F05C001501109A9
:100400002109310961F1908196239417B9F305C050
:10041000015011092109310911F19081962394139A
:10042000F7CFC12CD12CE12CF12C0AC08FEFC81AC8
:10043000D80AE80AF80A0C151D052E053F0579F0C3
:1004400080818623841791F36C2D7D2D8E2D9F2D19
:100450001F910F91FF90EF90DF90CF90089560E093
:1004600070E080E090E01F910F91FF90EF90DF909F
:10047000CF900895789484B5826084BD84B58160FE
:1004800084BD85B5826085BD85B5816085BD80915F
:100490006E00816080936E001092810080918100D7
:1004A00082608093810080918100816080938100CF
:1004B000809180008160809380008091B100846091
:1004C0008093B1008091B00081608093B0008091F2
:1004D0007A00846080937A0080917A0082608093B1
:1004E0007A0080917A00816080937A0080917A000E
:1004F000806880937A001092C10061E082E00E94DF
:10050000CD0060E084E00E94CD0061E083E00E94C5
:10051000CD0061E086E00E94CD0061E087E00E94AE
:10052000CD0061E088E00E94CD000AE8202E00E0C6
:10053000302ECEE9D0E060E082E00E94810083E0CE
:1005400090E00197F1F761E082E00E94810083E290
:1005500090E00197F1F760E082E00E948100EFE90E
:10056000F0E06491EBE8F0E08491E82FF0E0EE0F2A
:10057000FF1FE859FF4F8591949100E412E42FE0AA
:1005800030E0462F0E94F501611571058105910546
:1005900029F06F5F7F4F8F4F9F4F9F700E94AE0477
:1005A00026E933E44BE05DE30E94120520E030E0F1
:1005B00040E05FE30E9412050E9476049B01AC01BB
:1005C00020931301309314014093150150931601A9
:1005D00024363105410551050CF05FC168E873E12F
:1005E00080E090E00E94C90569017A0180910001D4
:1005F000833079F5E2E7F0E0149117FDEEC061E099
:1006000083E00E94CD00112309F492C0123009F05A
:100610009FC08091B100887F84608093B1002FEFEC
:100620003FEFA90109EFC114D104E104F10409F07D
:100630008CC00093B30020930701309308014093CE
:10064000090150930A0180917000826080937000CC
:10065000C4C08F3F09F0C1C083E080930001E2E78E
:10066000F0E014911F3F09F4B8C0113019F150F0B7
:10067000123009F43CC017FDB0C061E083E00E9475
:10068000CD00C4CF14BC15BC84B5826084BD85B5D3
:10069000816085BDF1018491E82FF0E0EE0FFF1F2E
:1006A000E358FF4F85919491FE0184918093060158
:1006B00010E0A5CF109280001092810080918100FF
:1006C00088608093810080918100816080938100A7
:1006D000F1018491E82FF0E0EE0FFF1FE358FF4F88
:1006E00085919491FE0184918093050188CF1092A9
:1006F000B0001092B1008091B00082608093B00091
:100700008091B10081608093B100F1018491E82F64
:10071000F0E0EE0FFF1FE358FF4F85919491909307
:10072000040180930301FE0184918093020167CF4D
:1007300085B5887F836085BD2FEF3FEFA90109EF65
:10074000C114D104E104F104D1F109EFB12C23C0AB
:100750001130B1F480918100887F816080938100A5
:100760002FEF3FEFA9010FE76EE3B62EC114D104BE
:10077000E104F10409F461C00FE78EE3B82E0BC069
:100780000FE79EE3B92E2FEF3FEFA901C114D1046B
:10079000E104F10461F0A8EEB3E0A70196010E9424
:1007A000E80528EE33E040E050E00E94A705113054
:1007B00009F443C0123009F43CCF11110EC007BD3B
:1007C00020930F01309310014093110150931201B7
:1007D00080916E00826080936E00C0901301D09073
:1007E0001401E0901501F0901601AAE0B0E0A70115
:1007F00096010E94E8054B015C010E94FE002B015E
:100800003C0181149104A104B10459F10E94FE003D
:100810006419750986099709683E73408105910539
:1008200080F3F1E08F1A9108A108B10828EE420E7A
:1008300023E0521E611C711CE4CF802F9B2D9093EE
:1008400089008093880020930B0130930C01409322
:100850000D0150930E0180916F00826080936F00B4
:10086000BCCF83E00E94230160E086E00E9481000B
:1008700060E087E00E94810060E088E00E948100E3
:10088000D701C601C397A109B109C297A105B10556
:1008900060F461E086E00E94810080E090E0892BB6
:1008A00009F449CE0E94000046CED701C601459703
:1008B000A109B1094E97A105B10538F461E086E0C0
:1008C0000E94810061E087E0E6CFF5E1CF16D10418
:1008D000E104F10414F761E086E00E94810061E028
:1008E00087E00E94810061E088E0D5CF0E947D040E
:1008F0006894B1110C940C0508950E94F10488F0DD
:100900009F5798F0B92F9927B751B0F0E1F0660FD3
:10091000771F881F991F1AF0BA95C9F714C0B13014
:1009200091F00E940B05B1E008950C940B05672F20
:10093000782F8827B85F39F0B93FCCF38695779543
:100940006795B395D9F73EF490958095709561952C
:100950007F4F8F4F9F4F0895E89409C097FB3EF457
:1009600090958095709561957F4F8F4F9F4F9923FC
:10097000A9F0F92F96E9BB279395F695879577957A
:100980006795B795F111F8CFFAF4BB0F11F460FF3A
:100990001BC06F5F7F4F8F4F9F4F16C0882311F092
:1009A00096E911C0772321F09EE8872F762F05C0A6
:1009B000662371F096E8862F70E060E02AF09A9541
:1009C000660F771F881FDAF7880F9695879597F936
:1009D000089557FD9058440F551F59F05F3F71F02F
:1009E0004795880F97FB991F61F09F3F79F0879596
:1009F0000895121613061406551FF2CF4695F1DF1F
:100A000008C0161617061806991FF1CF86957105AE
:100A1000610508940895E894BB2766277727CB01E2
:100A200097F908950E9425050C9496050E94880563
:100A300038F00E948F0520F0952311F00C947F056B
:100A40000C94850511240C940C050E94E90470F3A4
:100A5000959FC1F3950F50E0551F629FF001729F63
:100A6000BB27F00DB11D639FAA27F00DB11DAA1F72
:100A7000649F6627B00DA11D661F829F2227B00DBF
:100A8000A11D621F739FB00DA11D621F839FA00D4A
:100A9000611D221F749F3327A00D611D231F849F9A
:100AA000600D211D822F762F6A2F11249F575040F1
:100AB0009AF0F1F088234AF0EE0FFF1FBB1F661F6C
:100AC000771F881F91505040A9F79E3F510580F035
:100AD0000C947F050C940C055F3FE4F3983ED4F32F
:100AE000869577956795B795F795E7959F5FC1F7D9
:100AF000FE2B880F911D9695879597F9089597F984
:100B00009F6780E870E060E008959FEF80EC0895B3
:100B100000240A94161617061806090608950024DC
:100B20000A9412161306140605060895092E039456
:100B3000000C11F4882352F0BB0F40F4BF2B11F4CA
:100B400060FF04C06F5F7F4F8F4F9F4F0895A1E2FA
:100B50001A2EAA1BBB1BFD010DC0AA1FBB1FEE1F37
:100B6000FF1FA217B307E407F50720F0A21BB30B82
:100B7000E40BF50B661F771F881F991F1A9469F7FE
:100B800060957095809590959B01AC01BD01CF015A
:100B90000895052E97FB1EF400940E94E00557FD72
:100BA00007D00E94A70507FC03D04EF40C94E00583
:100BB00050954095309521953F4F4F4F5F4F089589
:100BC00090958095709561957F4F8F4F9F4F0895B9
:100BD0000E94F305A59F900DB49F900DA49F800DDA
:100BE000911D11240895A29FB001B39FC001A39F3E
:100BF000700D811D1124911DB29F700D811D112456
:080C0000911D0895F894FFCF47
:020C0800FF00EB
:00000001FF
